:020000021000EC
:10E000007EC00000BFC00000A3C00000A1C000008F
:10E010009FC000009DC000009BC0000099C0000090
:10E0200097C0000095C0000093C0000091C00000A0
:10E030008FC000008DC000008BC0000089C00000B0
:10E0400087C0000085C0000083C0000081C00000C0
:10E050007FC000007DC000007BC0000079C00000D0
:10E0600077C0000075C0000073C0000071C00000E0
:10E070006FC000006DC000006BC0000069C00000F0
:10E0800067C0000065C0000063C00000BBBEEC2D8F
:10E09000FD2DB7B6B0FCFDCF27BFE895B7B6B0FCF5
:10E0A000FDCF21E1B7B6B6FCF4CF0895040309040F
:10E0B0001C037700770077002E006600690073006C
:10E0C000630068006C002E00640065000E035500BC
:10E0D0005300420061007300700012011001FF0044
:10E0E0000008C016DC05020101020001090212004D
:10E0F000010100803209040000000000000011242A
:10E100001FBECFEFD0E4DEBFCDBF34B7D0E4CEEF3B
:10E110002991203F299109F02FEF20933F0130935F
:10E12000400111E0A0E0B1E0E2EAF9EE01E00BBF4E
:10E1300002C007900D92A630B107D9F711E0A6E012
:10E14000B1E001C01D92AF33B107E1F79FD127C401
:10E1500057CFA82FB92F80E090E041E050EA6095BA
:10E1600030E009C02D9182279795879510F084277C
:10E170009527305EC8F36F5FA8F30895EADF8D93AB
:10E180009D930895CF93CFB7CF93DF93C395499BCA
:10E19000E9F7499B0BC0499B09C0499B07C0499BB4
:10E1A00005C0499B03C0499B01C089C06F93C091C2
:10E1B0002201DD27C75DDE4F2F9365E5499B03C034
:10E1C0002F916F91E6CF0F931F934F9320E040E183
:10E1D0005F9309B1067001FB27F93F9350E03BE0E4
:10E1E00039C0167040642F77012F5F5F1EC04068F2
:10E1F00019B116702F7752501FC0406409B12F77A4
:10E200000670D1F15F5F00C023C0406219B12F7763
:10E21000167091F15F5F00C025C006701027515045
:10E2200012F45D5F0000115027952C3F19B1C8F61C
:10E2300016700127015027952C3FC8F642274993B5
:10E2400009B1067010274F73115027952C3FA8F67F
:10E250004695469519B1167079F00127015027951A
:10E260002C3F98F66B5A60F3315009B1B0F600C0FC
:10E2700011E01CBB002717C03B503195C31BD04099
:10E2800011E01CBB0881033CF9F00B34E9F020914C
:10E2900020011981110F1213EDCF093651F10D3202
:10E2A00011F0013E39F7009327013F915F914F91A3
:10E2B0001F910F912F916F91CCB3C0FD67CFDF916C
:10E2C000CF91CFBFCF91189520912701222369F3D9
:10E2D00010912501112339F534303AF1309325019D
:10E2E00020932101109122013BE0311B3093220148
:10E2F0001CC0009125010130B4F40AE53091000101
:10E3000034FD14C000930001C5E1D1E013C005271E
:10E3100010E000C000000BB91AC0052710E0221F52
:10E320001DC010E021C04AE502C032ED432FC4E118
:10E33000D0E032E01AB11660599A0BB11AB956E022
:10E3400020E865E320FF05270BB9279517951C3FAB
:10E35000F0F66695B8F7B1F720FF05270BB92795BA
:10E3600017951C3FD0F62795179517FF0527000036
:10E370001C3F0BB9B0F629913A9519F7097F109116
:10E380002601110FC651D0400BB911F01093200196
:10E3900011E01CBB02601AB1197F402F497F54E085
:10E3A0005A95F1F70BB91AB94BB97FCFFB01A89574
:10E3B00031978040E1F70895DC0113963C91139763
:10E3C0001496EC91149712962C911297203331F4F5
:10E3D000E370F0E0EE5FFE4F80810895932F8E2F63
:10E3E000283549F4332391F4E1E0F0E089E08093AB
:10E3F0005700849108952035E1F4332389F4E0E057
:10E40000F0E089E08093570084910895383009F056
:10E4100036C0E3E0F0E089E08093570084910895EE
:10E42000383069F5E2E0F0E089E0809357008491AC
:10E430000895203251F4A0E0B0E0880F991FAA1F80
:10E44000BB1FABBFFC0187910895283269F4A0E09F
:10E45000B0E0880F991FAA1FBB1F0196A11DB11D17
:10E46000ABBFFC0187910895203A09F46AC2203CB1
:10E4700021F415966C9172D202C02F3F11F080E00A
:10E48000089581EF80930B0180E008951AB881E030
:10E490008BB985BF82E085BF60E071E787DF04B696
:10E4A00003FE0EC08EEF9FE054D210E0805B904BD5
:10E4B00009F411E08EEF9FE06FEF7FEF5DD208C0AF
:10E4C00004B601FC02C010E003C019B11095117030
:10E4D00014BE112309F427C28EEF80930B0114BEE2
:10E4E00088E10FB6F89480936000109260000FBE30
:10E4F00080916900826080936900E89A519A8CE06B
:10E5000060E075E353DF5198789481EF80930B01BD
:10E5100090912501935097FD52C180912201CCE04A
:10E52000D0E0C81BD109C75DDE4F809121018D323B
:10E5300009F0C2C0983009F040C183EC8093150106
:10E540008AE58093000110920A013881832F80763A
:10E550002981882309F441C086E091E09093240149
:10E5600080932301233031F4CE0126DF809309010B
:10E5700024E098C0253079F12A3069F1822F845047
:10E580008630E0F48A819B8190930D0180930C0189
:10E59000293039F48C819D8190930F0180930E0175
:10E5A00018C08E81809310018D818270809311013B
:10E5B0002093120137FD71C09FEF70C0223021F40B
:10E5C00080910B018E7F03C080910B01816080934D
:10E5D0000B0120E067C021E065C08A8110921E0116
:10E5E000222331F410921F018EE191E022E050C00D
:10E5F000253019F48093260148C02630B1F58B816F
:10E60000813019F48AED90EE04C0823041F48CEE32
:10E6100090EE909324018093230122E122C0833065
:10E62000F9F48A81882341F48CEA90EE90932401D6
:10E630008093230124E015C0813041F480EB90EEFB
:10E6400090932401809323012CE10BC0823041F48C
:10E650008CEC90EE90932401809323012EE001C076
:10E6600020E080E480930A011DC0283019F488E27C
:10E6700091E009C0293019F48093280106C02A309E
:10E6800021F48EE191E021E003C08EE191E020E0F1
:10E69000909324018093230105C09E8180E880939C
:10E6A0000A0107C08F81882319F49E81921708F010
:10E6B000922F9093010181C080910A0187FF7DC054
:10E6C00080911001092F891708F4082F801B80936F
:10E6D0001001FF24882311F4FF24F39410E066C096
:10E6E00080911201873070F080910C0190910D01A2
:10E6F000019690930D0180930C01019769912ED1A1
:10E700001F5F54C040910C0150910D0160910E01AA
:10E7100070910F01403080EE580781E0680780E07B
:10E72000780708F048C01E5FF8948991999121E01C
:10E730000C01FA0160935B0020935700E8951124C7
:10E740007894DB01CA010296A11DB11D80930C01D2
:10E7500090930D01A0930E01B0930F01882341F017
:10E76000FF2021F1101710F1809111018823F1F0A1
:10E77000F89483E0FA0160935B0080935700E8957A
:10E78000789407B600FCFDCFF89485E0FA01609319
:10E790005B0080935700E895789407B600FCFDCFA6
:10E7A000F89481E180935700E8957894101708F465
:10E7B00097CFFF2011F01092010110922501809156
:10E7C000000184FF8CC0809101018F3F09F487C054
:10E7D000182F893008F018E0811B80930101809187
:10E7E000150198E8892780931501112309F465C064
:10E7F00080910A0187FF3DC080911001811708F4C4
:10E80000182F811B8093100100911201C6E1D1E005
:10E8100028C0073030F080910C0190910D0191D00B
:10E820000BC080910C0190910D01A0910E01B0914F
:10E830000F01ABBFFC0187918883219680910C0169
:10E8400090910D01A0910E01B0910F010196A11DB3
:10E85000B11D80930C0190930D01A0930E01B09314
:10E860000F01812F90E08A5E9E4FC817D90789F665
:10E8700022C0C0912301D091240186FF11C0212F15
:10E8800046E151E0CE01A0E0B0E0A160ABBFFC01E9
:10E890008791FA018193AF012196215099F707C022
:10E8A000912FE6E1F1E0899181939150E1F7D093C6
:10E8B0002401C0932301193060F486E191E0612FB7
:10E8C0005DDC612F6C5F6C3041F08FEF8093010154
:10E8D00004C08FEF809301016EE16093000194E129
:10E8E00089B1867031F49150D9F7109226011092B7
:10E8F000200180910B01803130F0489B0FC0809146
:10E900000B01805109C0489909C080910B018230E8
:10E9100028F080910B01825080930B0180910B01B4
:10E92000882309F0F5CDF894519A1BB81DBA1092BE
:10E93000690081E085BF15BEE0911301F0911401DB
:10E940000995F999FECF92BD81BDF89A992780B5B6
:10E950000895A8E1B0E042E050E013C0262FF999F5
:10E96000FECF1FBA92BD81BD20BD0FB6F894FA9AB2
:10E97000F99A0FBE01960895F1DF272FF0CFDC0141
:10E98000CB01FC01F999FECF06C0F2BDE1BDF89ABA
:10E99000319600B40D9241505040B8F70895F89464
:02E9A000FFCFA7
:06E9A2005AFF1E9705005C
:040000031000E00009
:00000001FF
